:020000040000FA
:040000008A01032846
:0A00060083120313981383160313EB
:1000100007309C009D019B011E30850086018312E4
:10002000031386010510831203132030A000103043
:10003000831203178C008D01831203135520831242
:1000400003178C0A8D0A83120313A00B1E2820307D
:10005000A000831203178D014D2083120313860025
:100060004920831203178D0A83120313A00B2C2837
:1000700063001930A200A100A10B3C28A20B3B2871
:100080000800FA30A200A100A10B4428A20B4328CB
:1000900008004120412041200800831603178C13DB
:1000A0000C14831203170C080800831603178C1313
:1000B0000C158B1355308D00AA308D008C148C18C4
:0800C0005F280C118B170800EA
:00000001FF
